:020000040000FA
:10000000A0040020352900003D2900003F29000000
:1000100000000000000000000000000000000000E0
:100020000000000000000000000000004129000066
:1000300000000000000000004329000045290000E6
:1000400047290000472900004729000047290000F0
:1000500047290000472900004729000047290000E0
:1000600047290000472900004729000047290000D0
:1000700047290000472900004729000047290000C0
:1000800047290000472900004729000047290000B0
:1000900047290000472900004729000047290000A0
:1000A0004729000099020000472900004729000065
:1000B0004729000047290000472900004729000080
:1000C00000F002F800F0BDF80CA030C80838241881
:1000D0002D18A246671EAB4654465D46AC4201D180
:1000E00000F0AFF87E460F3E0FCCB64601263342F5
:1000F00000D0FB1AA246AB463343184730440000F9
:1001000050440000103A02D378C878C1FAD8520798
:1001100001D330C830C101D504680C6070470000BD
:100120000023002400250026103A01D378C1FBD813
:10013000520700D330C100D50B60704710B56E294F
:1001400002D102F075FD10BD702902D102F0B7FE98
:1001500010BD662902D104F0D5F810BD652902D181
:1001600004F0D0F810BD672902D104F0CBF810BD1F
:10017000612902D1C046C04610BD03681B0A01D3E5
:1001800080231943692902D102F01CFD10BD6429A6
:1001900002D102F017FD10BD752902D102F012FD47
:1001A00010BD6F2902D102F035FE10BD782902D1B1
:1001B00002F072FE10BDE92902D102F0D1FD10BD9E
:1001C000E42902D102F0CCFD10BDF52902D102F0E4
:1001D000C7FD10BDEF2902D102F028FE10BDF8299D
:1001E00002D102F067FE10BD0368DB0901D3802352
:1001F0001943632902D103F0E0F910BD732902D13C
:1002000003F0E3F910BDE32902D103F0EDF910BDCD
:10021000F32902D103F0F0F910BD002010BD1FB585
:1002200003F04AFA04000020002104F055F8401CB5
:1002300060600020002104F039F8E0601FBD10B5B7
:1002400010BD03F011FA1146FFF7E9FF00F025F8A1
:1002500003F0A6FD03B4FFF7F2FF03BC03F0F0FDCB
:1002600070B505460C46164602E00FCC0FC5103E91
:10027000102EFAD2082E02D303CC03C5083E042E5A
:1002800007D301CC01C5361F03E021782970641C17
:100290006D1C761EF9D270BD704700BF00BF00BF55
:1002A00059204E49086016200860882008600846DA
:1002B00000680028F4D000BF00F0B1F800BF0020B3
:1002C0004649086000BF382000F060FC00F0EFFBFA
:1002D00000F0FDFB424840680721090608434049F9
:1002E000486000F000FB0221002000F04EFB0321DB
:1002F000022000F04AFB0421084600F046FB00F013
:1003000047FA00F039FC374800F01EFC36490878FF
:1003100000F03CFC35490D68E90F49194910344A91
:1003200088183249096802F03BFB441E2146002030
:1003300000F080FA2146022000F07CFA21460420D9
:1003400000F078FA2BA000F09BFC46E003F086FE5C
:1003500000BF2A488068C007C00F00283DD000BFFA
:1003600001202649886000BF25480068002801D187
:1003700003F06EFD00F0B9FD00282ED02048006883
:1003800001280FD1452000F001FC0021084600F0B3
:1003900051FA0021022000F04DFA0021042000F063
:1003A00049FA1AE0302000F0F1FB10490D68E90F1E
:1003B000491949100E4A88180C49096802F0F0FAE8
:1003C000441E2146002000F035FA2146022000F0AC
:1003D00031FA2146042000F02DFAB7E70001005061
:1003E0000000044020A107000800002000000020B9
:1003F00000A24A040D0A4F4B2000000000010140FA
:100400001400002000BF5920F94908601620086038
:1004100088200860084600680028F4D0704710B5AE
:10042000042001F0DFFD102001F03CFC002107203A
:1004300001F048FC012001F0D5FD012001F032FC63
:10044000EC4801F01FFD042001F02CFCEA4801F00B
:10045000D5FD00221146E84801F05CFDE74801F0B7
:10046000CDFD032252040C21E44801F053FDE44881
:1004700001F0C4FDE34801F0C1FDE34801F0BEFD19
:10048000002201214902E04801F044FDDF4801F06B
:10049000B5FD002201214903DC4801F03BFDDC48A9
:1004A00001F0ACFD002201214904D94801F032FDE0
:1004B000D84801F0A3FD002201210907D04801F02E
:1004C00029FD002201214907CE4801F023FDD24831
:1004D00001F034FBD048401C01F030FB0520000740
:1004E000406B000A00020521090748630846406B7B
:1004F000332108430521090748630846806B000E35
:10050000000688630846806BC44908430521090733
:100510008863B748C038806800090001B449C03911
:1005200088600846806805210843B149C039886061
:10053000084680680F2109038843AD49C0398860A7
:100540000846806809140843A949C0398860002218
:100550004021B34802F036F9A548C03800680009C8
:100560000001A349C0390860084600680621084315
:100570009F49C039086008460068F02188439C49BB
:10058000C039086008460068602108439849C039AE
:100590000860084600680F21090288439449C03961
:1005A0000860084600680321490208439049C039A1
:1005B0000860084600680F21090388438C49C03948
:1005C0000860084600680321490308438849C03988
:1005D0000860084600680F21090488438449C0392F
:1005E0000860084600680321490408438049C0396F
:1005F0000860084600680F21090588437C49C03916
:100600000860084600680321490508437849C03955
:100610000860084600680F21090688437449C039FC
:100620000860084600680321490608437049C0393C
:10063000086005200007C06B0F21090488430521CD
:100640000907C8630846C06B032149040843052114
:100650000907C8630846006B0F2109038843052179
:10066000090708630846006B032149030843052175
:10067000090708630846006B0F210902884305211A
:10068000090708630846006B032149020843052156
:10069000090708630846006BF02188430521090714
:1006A00008630846006B60210843052109070863B9
:1006B0000846006B0009000108630846006B06212C
:1006C000084305210907086303221021544880309C
:1006D00002F078F8032220215148803002F072F8AD
:1006E000032240214E48803002F06CF80322802122
:1006F0004B48803002F066F80322042148488030DD
:1007000002F060F803220121C902454802F05AF8BC
:100710000322FF2101314248803002F053F80322C6
:10072000012149023E48803002F04CF803220121A9
:1007300089023B48803002F045F803220121C902BA
:100740003748803002F03EF8032201210903344883
:10075000803002F037F8032201214903304880300D
:1007600002F030F80322012189032D48803002F085
:1007700029F803220121C9032948803002F022F818
:100780000322012149022648403002F01BF810BD27
:1007900010B5244800680121084322490860224B13
:1007A0000C2200211F48803800F02CFC01201D493C
:1007B0000861084600680121C90208431949086018
:1007C00010BD10B5062807D2184B84001A51174BDC
:1007D00020338400195109E00C2807D2801F144BE4
:1007E00084001A51124B20338400195110BD0000AF
:1007F0000001005000A24A04113D80571CFE235600
:100800001400C0531500D0530200805E0300C05E88
:100810000400005F1E0000401400000411111100CC
:100820004040005080000E403F4000003000044037
:100830003000144006280FD240084000FA4A8300D6
:10084000D150431C9B00D1504908F74A2032830005
:10085000D150431C9B00D150704706280FD240084E
:100860004000F24A8300D150431C9B00D1504908FC
:10087000EE4A20328300D150431C9B00D150704778
:1008800010B500234A0894000246143213514B005D
:1008900003229A4001231B048B401A43436893436D
:1008A0004360E34B8C0002463032135100238C002E
:1008B00020321351B02212584C00DE4BA3409A4311
:1008C0004C000223A3401A43B0231A50B4221258FA
:1008D0004C00D84BA3409A434C000123A3401A4339
:1008E000B4231A5010BD10B50021CF483038FFF79F
:1008F000C7FF0121CC483038FFF7C2FF0221CA48A8
:100900003038FFF7BDFF0321C7483038FFF7B8FF85
:100910000421C5483038FFF7B3FF0521C2483038FD
:10092000FFF7AEFF3F21C048303800F07BFE3F218B
:10093000BD48303800F02EFD0021BC483038FFF7AC
:100940009FFF0121B9483038FFF79AFF0221B748CD
:100950003038FFF795FF0321B4483038FFF790FF98
:100960000421B2483038FFF78BFF0521AF483038FB
:10097000FFF786FF3F21AD48303800F053FE3F219E
:10098000AA48303800F006FD10BD70B505460C468B
:10099000FFF738FDA848844200D904462B0003F035
:1009A00059FC060405161726273600BF9E4810304E
:1009B000006B01210906884340189B4910310863E8
:1009C000224600219848303800F05EFE1FE000BF4C
:1009D00095483038406F01210906884341189248F4
:1009E000303841672246022100F04EFE0FE000BF82
:1009F0008D483038806F01210906884341188A48A4
:100A0000303881672246042100F03EFE00BF00BF5F
:100A100000BF00208949086000BF70BD70B5054661
:100A20000C46FFF7EFFC8448844200D904462B00B3
:100A300003F010FC060405161726273600BF7B4876
:100A40001030006B012109068843401877491031A6
:100A50000863224600217548303800F015FE1FE07B
:100A600000BF72483038406F0121090688434118A1
:100A70006E48303841672246022100F005FE0FE043
:100A800000BF6A483038806F012109068843411849
:100A90006648303881672246042100F0F5FD00BF2A
:100AA00000BF00BF00206549086000BF70BD10B5E1
:100AB00064220021624801F099FD61480068000A43
:100AC000000247305E4908605E48486010BD10B5BE
:100AD00064220121C9065C4801F088FD5A4800F0F3
:100AE0006EFA10BD10B5594A0121C906584801F0E7
:100AF0007DFD00BF5648006801214907084354495D
:100B0000086000BF084600F05AFA0021192000F0E2
:100B10001FFA0A20012181404E4A116000BF10BD1A
:100B200010B54D4A0121C9064C4801F05FFD4B4804
:100B30000068000A00024730484908604848486099
:100B4000084600F03CFA10BD70B5054600240CE0E4
:100B500000BF3D488068C007C00F002805D000BF17
:100B600001203949886000BF641C3E49284601F0D5
:100B700021FFA042ECDC70BD10B53B4800F0DEFF69
:100B8000E1214902394801F081FB10BD01462039BD
:100B9000374A505CC107C90F002903D00021354AEC
:100BA000116202E00121334A116202210140002951
:100BB00003D000212F4A516202E001212D4A5162E7
:100BC00004210140002903D000212A4A916202E059
:100BD0000121284A916208210140002903D0002107
:100BE000244AD16202E00121224AD162102101404F
:100BF000002903D000211F4A116302E001211D4A90
:100C0000116320210140002903D00021194A5163BA
:100C100002E00121174A51634021014000292BD0F5
:100C20000021144A91632AE030000440300014404F
:100C300000A24A0403000300FF0F0000000100505F
:100C400000000140CB2B0000000101408545010060
:100C50000000114000E100E040420F00000111409F
:100C6000FFFFFF00102700001100000400001540E6
:100C70002C430000C04200500121D44A91637047C8
:100C80000FB410B5A2B025A80190802102A8019B45
:100C9000249A01F069FE04460020019000BF0DE097
:100CA00000BFCB4989690122D2051140C90D002935
:100CB000F7D102A9095CC64A1160401CA042EFDBD3
:100CC00022B010BC08BC04B0184710B502460B4651
:100CD000D7E0BF480068C1B20D2901D00A2914D15C
:100CE000BC48006804280CDB0020BA4C2060BA48DD
:100CF000407830381060B94800681860B64800780D
:100D000010BD0020B34C2060BAE0202904D100209F
:100D1000B04C20602020F3E7612901D0412904D1A3
:100D20000020AC4C20606120EAE7772901D05729E8
:100D300004D10020A74C20607720E1E7642901D08E
:100D4000442904D10020A34C20606420D8E77829EE
:100D500001D0582904D100209E4C20607820CFE794
:100D6000462903D0542901D0562905D19A4801704B
:100D70000120984C206083E09648006801287FDBC2
:100D80009748944C2468005D6E2826D1302901DBF9
:100D9000392903DD00208F4C206071E08F48006806
:100DA0000A246043401830388C4C20608A48894CB3
:100DB0002468015587480068401C864C206006283E
:100DC0005ED300202060844840783038106083482B
:100DD000006818608048007892E781487D4C24685C
:100DE000005D6D2830D13F290BD10020794C206067
:100DF00079484078303810607748007820242043C4
:100E00007EE7302901DB392903DD0020714C2060A9
:100E100036E008463038714C20606F486D4C2468CD
:100E200001556C480068401C6A4C2060062827D396
:100E300000202060684840783038106067480068BB
:100E40001860654800785BE76548624C2468005D7F
:100E5000884212D15F480068401C5E4C2060062822
:100E60000ED3002020605C484078303810605B482A
:100E7000006818605848007842E70020554C206010
:100E800000BF53488069012189030840002800D130
:100E90001FE7002034E710B500231A46012151480E
:100EA00001F0C2FC4F484068C02188434D4948606A
:100EB000084640680721490388434018494948606B
:100EC000084640680121090308434649486008462E
:100ED0004068032109028843424948600846406847
:100EE000022108433F49486010BD3F48006881B275
:100EF0003E4881420ADB3E48006801280FD00120AD
:100F00003B4A106000203B4A106008E03848006807
:100F1000002804D00020364A1060364A1060354858
:100F200000680A2812D233480068401C314A106019
:100F30000A280BD1304800682D4A1268904205D02B
:100F40002B4800682C4A1060012070470020FCE705
:100F500010B5002819DA294A03071B0F083B9B0824
:100F60009B00D2588307DC0EFF23A3409A438B07D4
:100F70001B0E8407E40EA3401A43204B0407240FE2
:100F8000083CA408A4001A5118E01D4A03231B02C0
:100F9000D21883089B00D2588307DC0EFF23A3409E
:100FA0009A438B071B0E8407E40EA3401A43144B8D
:100FB000032424021B198408A4001A5110BD0168DF
:100FC000012292071143016070470000C0420050A7
:100FD00000001540240000201C0000201800002004
:100FE0008743000000000D4000000E404507000050
:100FF000100000200C000020140000201CED00E078
:1010000000E100E030B580242458494D2C400C43C9
:10101000144380252C508424245884252B5030BD23
:1010200005210907C9680122120711430522120789
:10103000D1601146C96801221207914305221207A7
:10104000D160704710B500290CD180231B58FF24B4
:10105000F134A3430B431343FF240134234380247F
:1010600023501EE010290AD180231B58FF24F1349D
:10107000A3430B430C0123438024235011E09C2302
:101080001B581B0A1B0213439C24235080231B580C
:10109000FF24F134A3430B43FF2401342343802472
:1010A000235010BD80210958FF22F1329143802244
:1010B00011507047CA07D20F002A05D0802212585B
:1010C00002231A4380231A5002220A40002A05D024
:1010D0008822125802231A4388231A5004220A40F5
:1010E000002A05D08C22125802231A438C231A504E
:1010F0007047CA07D20F002A05D080221258022357
:101100009A4380231A5002220A40002A05D08822DE
:10111000125802239A4388231A5004220A40002AB4
:1011200005D08C22125802239A438C231A50704700
:10113000F3FBFFFFFEB500200290FBA000680090CB
:10114000FA48046A00132040002801D00020FEBDA8
:101150000120C0042040002801D0F54D00E0F54DED
:10116000012040042040002801D02846EFE703205A
:1011700080032040800B69460A5C0192E005C00DA7
:10118000861C1F2040022040400A871C019A7A4397
:101190001146AA087243104601F002FC800002903A
:1011A0000298D4E7FFB583B004460D460127E24814
:1011B0000090E248844205D1DC484069A102084021
:1011C000029005E0D9484069012149070840029092
:1011D0000298002803D1FFF7ADFF06460BE001F0AF
:1011E00037FBD648844203D100F036FD064602E0C4
:1011F00000F042FD06467D21C900304601F0D0FBDB
:10120000064601271AE0CE4979430846314601F0E7
:10121000C7FB01900599019888420DD20120000377
:10122000874200D10EE0781CC549414301987043C4
:10123000814200D806E000E004E07F1C01200003AA
:101240008742E0D900BF781E074669088A00214618
:101250001431885060686A000321914088436A0015
:101260000121914008436060606801210904A940A0
:1012700088436060AA002146303100988850019868
:1012800007B0F0BDFFB585B004460D460126AA485B
:101290000290AA48844205D1A4484069A1020840AE
:1012A000049005E0A14840690121490708400490E5
:1012B0000498002803D1FFF73DFF07460BE001F03B
:1012C000C7FA9E48844203D100F0C6FC074602E0FC
:1012D00000F0D2FC0746012612E03846079901F0DB
:1012E0005FFB3146019001F05BFB03900121090493
:1012F0000398884200D902E00398029003E0761C2C
:1013000090488642E9D300BF0298704301463846B0
:1013100001F046FB0390701E064669088A002146CC
:101320001431885069000320884001210904A94034
:1013300008436168814361600298401EAA0021460B
:10134000303102908850029A521C08995143084645
:10135000642101F025FBAA00214650318850B020BD
:1013600000596A007849914088436A0002219140FF
:101370000843B0210851B42000596A0072499140D5
:1013800088436A00012191400843B4210851039821
:1013900009B0F0BD026A0A430262704730B50246E6
:1013A00000200AE0012383400B40002B04D00024DE
:1013B0008500134630335C51401C0628F2D330BD03
:1013C000026A8A430262704730B5042911D2F823B9
:1013D0001C58CD000F23AB409C43F8231C508023A6
:1013E0001343CC00A340F82424582343F82423506B
:1013F00012E0FC231B580C1FE5000F24AC40A34354
:10140000FC242350802313430C1FE400A340FC243E
:1014100024582343FC24235030BD10B5042908D29E
:10142000F8221258CC008023A3409A43F8231A5084
:1014300008E0FC2212580B1FDC008023A3409A43D3
:10144000FC231A5010BD10B501231B048B40FF2450
:101450002134235010BD0246FF2021308058012343
:101460001B048B401840002801D001207047002049
:10147000FCE7F0B504460020B6E0012585400D40AC
:10148000002D2FD0812B0CD0822B0AD0882B08D096
:101490002E4DAB4205D06D1CAB4202D0AD1DAB4210
:1014A00015D14508AE002546C835AD59274E7F36C3
:1014B0001E4035434608B6002746C837BD51C425EF
:1014C0002D591E07360F3543C42635510AE045080D
:1014D000AE002546C835AD591D434608B60027461F
:1014E000C837BD51012585401540002D48D0C5079E
:1014F000ED0F002D2CD14508AE002546C835AD595D
:1015000003263604B5434608B6002746C837BD5102
:101510004508AE003D46AD5903263604354346081E
:10152000B600BD515FE0000001020204000200505D
:1015300000805101001BB700FFFF000000000440C5
:1015400040420F00FF0F0000030003000180000075
:101550004508AE002546C835AD590326B604B54347
:101560004608B6002746C837BD514508AE003D467F
:10157000AD590326B60435434608B600BD5132E0E6
:10158000C507ED0F002D17D14508AE002546C8351B
:10159000AD5903263604B5434608B6002746C8377A
:1015A000BD514508AE003D46AD5901267604354390
:1015B0004608B600BD5116E04508AE002546C835C0
:1015C000AD590326B604B5434608B6002746C837CA
:1015D000BD514508AE003D46AD590126F6043543E0
:1015E0004608B600BD51401C062800D245E7F0BDB4
:1015F0000122520212580A4301235B021A501A1D9B
:1016000012580A431B1D1A507047012252021258E9
:101610008A4301235B021A501A1D12588A431B1D6C
:101620001A507047D82212580A43D8231A507047CC
:10163000D82212588A43D8231A507047F0B5CC07E5
:10164000E40F8F25AD002D584E08F7001E26BE4032
:10165000B5432601D7003E431E4301273E434F08B2
:10166000FF00BE4035438F26B6003550F0BD10B5A3
:101670008F22920012584B08DC000123A3409A43AA
:101680008F239B001A5010BD30B54B089C000346B9
:1016900070331B591C0B24034B089D000346703309
:1016A0005C514B089C00034670331B5901242404F1
:1016B000144323434C08A50004467034635130BDE5
:1016C00010B54A08930002467032D25801231B0419
:1016D0009A434B089C00034670331A5110BD10B555
:1016E00025231B011B5814468C4023432524240129
:1016F000235010BD10B525231B011B5814468C40E8
:10170000A34325242401235010BD10B513468B405C
:101710009524A400235010BD10B5024695208000EA
:101720008058FF2301338B401840002801D001204E
:1017300000E00020400095239B009B5801248C4032
:101740002340002B01D0012300E00023184310BDEB
:1017500010B5E0231B5814468C402343E02423504B
:1017600010BDE0221258DE4B8B409A43E0231A5002
:101770007047DB4A8A40E8231A5070470246E82047
:101780008058D74B8B401840002801D0012070476B
:101790000020FCE7E422125807238B401A43E4237D
:1017A0001A507047E422125807238B409A43E423CF
:1017B0001A5070473F228A40EC231A507047024665
:1017C000EC2080583F238B401840002801D0012096
:1017D00070470020FCE710B5E0231B58FF240134BC
:1017E0008C402343E024235010BDE0221258FF23F5
:1017F00001338B409A43E0231A507047FF22013295
:101800008A40E8231A5070470246E8208058FF2398
:1018100001338B401840002801D001207047002080
:10182000FCE7E022125801238B401A43E0231A50B0
:101830007047E022125801238B409A43E0231A504C
:10184000704701228A40E8231A5070470246E82078
:10185000805801238B401840002801D00120704798
:101860000020FCE770B5F02424584D08EE007F25D9
:10187000B540AC431D018026354315434E08F600A4
:10188000B5402C43F0252C5070BD10B5F0221258F5
:101890004B08DC008023A3409A43F0231A5010BD6C
:1018A00010B5E02212584B08DC008023A3401A43F5
:1018B000E0231A5010BD10B5E02212584B08DC008E
:1018C0008023A3409A43E0231A5010BD4A08D30056
:1018D00080229A40E8231A50704710B50246E8204B
:1018E00080584B08DC008023A3401840002801D01A
:1018F000012010BD0020FCE74B08FF2202329A4075
:1019000003231B02C318DA64704710B50246032094
:1019100000021018C06C4C08FF230233A34018408B
:10192000002801D0012010BD0020FCE710B503689D
:1019300014468C402343036010BD10B50368144661
:101940008C40A343036010BDF0B5059C49084E00D0
:1019500003252D02B540012636068E402E438568AC
:10196000B5431E068E40354316024F00BE40354338
:1019700085608D00064680367451F0BD30B5024654
:1019800000200BE0012383400B40002B05D093681F
:1019900045080124AC4023439360401C0628F1D342
:1019A00030BD30B5024600200BE0012383400B40E0
:1019B000002B05D0946845080123AB409C439460FC
:1019C000401C0628F1D330BD30B50B055404234329
:1019D000012424041B1984683F256D04AC43234370
:1019E000836030BD81680122120491438160704799
:1019F00081680122D205114381607047816801220C
:101A0000D20591438160704730B503694C08E50009
:101A10000724AC40A3434C08E5001446AC402343E4
:101A2000036130BD70B5C0242458CE007E25B5407A
:101A3000AC4315015E0035436D1CCE00B5402C4310
:101A4000C0252C5070BD10B5C0221258CC00012307
:101A5000A3409A43C0231A5010BD10B5C02212589B
:101A6000CC008023A3401A43C0231A5010BD10B5E8
:101A7000C0221258CC008023A3409A43C0231A509E
:101A800010BD30B5C0231B58CD0001242404AC4048
:101A9000A343CC0010341546A5402B43C02423504B
:101AA00030BD70B5049C15460D432543FF261936FD
:101AB00035505D1E361D355070BD0246FF20213069
:101AC000805801238B401840002801D00120704726
:101AD0000020FCE701228A40FF2321331A5070477F
:101AE0000000010105210907486070470520000733
:101AF0008069402108408009704705200007406840
:101B000070472B480068C007C00F0121484070474C
:101B10000520000700687047052000078068012144
:101B20000843052109078860704705200007806881
:101B3000022108430521090788607047010E05222C
:101B4000120789188968012282401143020E052379
:101B50001B07D2189160010E1A4689188A68012164
:101B600081408A43010EC9188A6070470522120716
:101B7000926901231A4305231B079A611A46926949
:101B800008239A43024305231B079A611A46926968
:101B900006239A430A4305231B079A6170470520D1
:101BA00000078069400840000521090788617047E7
:101BB00000010050F648806840218843F44988605D
:101BC000704710B510230B4354012343F04C63625C
:101BD00023469B6840242343ED4CA3602346DB69E6
:101BE0001C24A3430343EA4CE36110BDE9480069A8
:101BF00004210843E7490861E5480068802108435B
:101C0000E349086030BF7047E24800690421884317
:101C1000E0490861DE48006880218843DC490860AB
:101C200030BF7047DA480068C007C00F002801D0F5
:101C3000D94870470020FCE7D548006802210840D9
:101C4000002801D0880370470020FCE710B500F0A1
:101C5000FFFDD248006810BD10B500F0F9FDCC487A
:101C6000006940210840002803D0CC4800684008A3
:101C700010BDCA480068FBE710B500F0E9FDC44894
:101C8000006980210840002803D0C448006840084B
:101C900010BDC2480068FBE710B500F0D9FDBF4891
:101CA000006810BD0146BE4A05E01046521E0028DD
:101CB00001DC00207047B648C06808408842F4D173
:101CC0000120F7E770B504460D46B148C068102101
:101CD00008400646AE48006804210843AC49086045
:101CE0001020FFF7DFFFAA480069C008C000C01D30
:101CF000A7490861084680690009000128438861F6
:101D000008460069C008C0002043086100F0A0FD3B
:101D1000002E05D19E480068042188439C49086034
:101D200070BD9B48006A0121090408439849086274
:101D30007047F3B589B00C46FFF7F3FF0998002808
:101D40000ED19348006801210843914908600120A1
:101D5000FFF7A8FF002006908F48089002250EE0AC
:101D60008B48006804210843894908601020FFF768
:101D700099FF0120C00406908A48089004258A48EB
:101D8000844204D84010844201D9002712E08748D9
:101D9000844205D84010844202D90127640009E03A
:101DA0008348844205D84010844202D30327A4000C
:101DB00000E057E00020C043039000200190029013
:101DC00034E02946089800F0EBFD05907949059824
:101DD00088422AD978490598884226D2022007905D
:101DE0001EE0059E07994E437048864215D3400079
:101DF000864212D8A64201D9301B00E0A01B0490F5
:101E000003990498884208D2049803900195079892
:101E100002900398002800D106E00798401C079024
:101E2000664907988842DCD900BF6D1C212DC8D9AE
:101E3000B803069908430199891E4902084302998B
:101E4000891E0843524908620420FFF72BFF781CC3
:101E5000019A50430146089800F0A2FD02994843B8
:101E60000BB0F0BD0998002803D1554848490862D5
:101E700002E05448464908620420FFF713FF00F0CF
:101E800019F9EDE770B504464148C06810210840D3
:101E900005464D48844200D904464C48844200D24D
:101EA00004463B4800680421084339490860102073
:101EB000FFF7F8FE364800690721084334490861F6
:101EC000084680690009000188610846C068C007AB
:101ED000C00F002805D061000020FFF72AFF04464C
:101EE0000AE061000120C004FFF723FF04462848F0
:101EF000C06810210840054601210220FFF7E2FEDC
:101F0000002D05D12248006804218843204908603B
:101F1000600870BDF7B586B0002200232C4C254622
:101F2000E0CDE4680497039602950594284D10359A
:101F300030CD019500948403240E002C11D00403AD
:101F4000A40FA4006D462C59114D18356319840354
:101F5000250E8405E40EA5401C68AC43089D2C4367
:101F60001C600401640F002C10D08400A40FA40096
:101F700002AD2C59064D103562190401650FC401DC
:101F8000E40EA5401468AC430C43146009B0F0BDE6
:101F90000002005000ED00E0001BB7002800002008
:101FA00080F520000080510100C2EB0B00E1F50537
:101FB00080F0FA02006A18000024F4000102000018
:101FC0002E440000324C080000A24A0440787D01F3
:101FD0009043000053490969382291430143514A13
:101FE000116170474F49096801434E4A11607047BB
:101FF0004C49096881434B4A116070470EB54A4B02
:102000001A6859689B68029300920191810F8900B8
:102010006A465158434A89184968C306DB0E0122B3
:102020009A401143820F92006B469A583D4BD2184A
:1020300051600EBD0EB53C4B0C331A6859689B6855
:10204000029300920191810F89006A465158354AE6
:1020500089184968C306DB0E01229A409143820F1A
:1020600092006B469A582F4BD21851600EBD002239
:102070002E4B1A61042806D11A46126904231A430A
:102080002A4B1A6106E0274A126938239A43024311
:10209000244B1A61254A51610022244B9A611A4649
:1020A000126903231A43214B1A61704700201F490C
:1020B00008617047FEB5002002901DA000680090E6
:1020C0001848046A00132040002801D00020FEBDFB
:1020D0000120C0042040002801D0164D00E0164D1C
:1020E000012040042040002801D02846EFE70320CB
:1020F00080032040800B69460A5C0192E005C00D18
:10210000861C1F2040022040400A871C019A7A4307
:102110001146AA087243104600F042FC800002906B
:102120000298D4E700020050A843000000E000E05D
:102130000102020400805101001BB700FEB500201F
:102140000290FBA000680090FA48046A0013204047
:10215000002801D00020FEBD0120C004204000283E
:1021600001D0F54D00E0F54D01204004204000284D
:1021700001D02846EFE7032080032040800B69460A
:102180000A5C0192E005C00D861C1F204002204021
:10219000400A871C019A7A431146AA0872431046E6
:1021A00000F0FEFB800002900298D4E70122920228
:1021B0000A40002A01D0682282610122D2020A402C
:1021C000002A03D0426901231A43426101225203CB
:1021D0000A40002A01D0DA4A8261012292030A40B1
:1021E000002A01D0426C42640122D2030A40002A34
:1021F00003D08022C261826B8263704700214160FC
:10220000704741680322120391434160704770B5E3
:1022100004460D466068A8436060CA48844203D102
:102220000C2000F0A2F909E0C748844203D10D2038
:1022300000F09BF902E00C2000F097F970BD0169F5
:10224000012252021143016141695210114341615F
:1022500041680322120311434160704770B5044680
:102260000D46606828436060B648844203D10C2064
:1022700000F074F909E0B448844203D10D2000F065
:102280006DF902E00C2000F069F970BDF0B587B07F
:1022900004460D46AD4801460EC9C06803AE0EC6E1
:1022A000069000200290A3484069032109060840D7
:1022B000060EA04880690F2109020840070A002085
:1022C00020630320E060A068A1490840A060012EBF
:1022D00004D1FFF733FFB10003AA5050002D26D0E0
:1022E000B10003AA5058791C00F05AFB6908401845
:1022F0002946019000F054FB801E029095490298F7
:1023000088420FD9B10003AA5058791C00F048FB4D
:10231000E90040182946019000F042FB0009801EA8
:10232000606204E00321090702980843606207B075
:10233000F0BD70B503460C46002111E0002506E013
:102340006D1C01208007854201D3002070BD986973
:102350000126B60330400028F2D118686054491CA9
:102360009142EBD30846F1E7FFB587B004460D462E
:1023700017467648103001460EC9C06802AE0EC638
:102380000590002001906B48406903210906084030
:10239000060E684880690F2109020840000A06906D
:1023A000012E04D1FFF7CAFEB10002AA5050002D41
:1023B00028D0B10002AA50580699491C00F0F0FA42
:1023C000690840182946009000F0EAFA801E019042
:1023D00060490198884210D9B10002AA5058069964
:1023E000491C00F0DDFAE90040182946009000F091
:1023F000D7FA0009801E606204E0032109070198F2
:102400000843606238460A99084310990843E0601F
:102410000BB0F0BD026A120A12020A43026242685D
:102420000123DB021A4342607047F7B586B00446C9
:102430000E464648203001460EC9C06801AD0EC5A3
:102440000490022020633B484069032109060840AC
:10245000070E384880690F2109020840000A0590DC
:10246000012F04D1FFF76AFEB90001AA5050002ED7
:1024700012D0B90001AA50580599491C00F090FAF1
:10248000F10040183146009000F08AFA0009851EDC
:102490003048854200D265620898002808D1A06AB9
:1024A00040210843A062A06A02218843A06207E09D
:1024B000A06A20218843A062A06A02210843A0628A
:1024C00009B0F0BD10B503230363C36A224C234057
:1024D000C362C36A14060C432343C36210BD10B524
:1024E00001230363C36ACF24A343C362C36A0C46B8
:1024F00014432343C36210BD70B503460C4600214C
:1025000011E0002506E06D1C01208007854201D303
:10251000002070BD98690126360730400028F2D0AF
:10252000605C1860491C9142EBD10846F1E700005D
:10253000010202040002005000805101001BB7009C
:10254000010000010000054000001540C0430000EC
:102550000FFFF0FFFFFF0000FFF8FF00C206D20EE2
:1025600001219140054A11607047C206D20E012137
:102570009140024A803211607047000000E100E0A3
:1025800030B589B005462022824901A8FDF768FED2
:102590008148854206D181484069072109020840E7
:1025A000040A19E07E48854206D17C48406907212B
:1025B00009030840040B0FE07A48854206D17748AA
:1025C0004069072109040840040C05E0734840698C
:1025D000072109050840040D022C03D17248006848
:1025E00009B030BDA00001A90858F9E7F7B582B0DD
:1025F000064617463046FFF7C3FF0190002400252A
:1026000001984008B84201D202240CE039460198F2
:1026100000F0C6F90446250E002D04D0691C2046A2
:1026200000F0BEF904460398284330607460681CCB
:1026300060430146019800F0B3F905B0F0BD0021F8
:10264000016041617047FEB505460C462846FFF71C
:1026500097FF07460020029039465348006800F073
:102660009FF9401C01900020286068614F48874214
:1026700009D87D20C000844200D204464B488442E1
:1026800008D9044606E0642C00D2642447488442FA
:1026900000D90446454887420FD8002002903946A9
:1026A000434800F07DF900907D21C9006143084650
:1026B000009900F075F9064610E03C49384600F0F4
:1026C0006FF906466643300E02900298002805D046
:1026D0000299491C304600F063F906466E600121FC
:1026E000890702980843286003E000BF0198401E54
:1026F000019001980028F8D100BF286801214906FF
:1027000008400028F9D1FEBD10B54369294C23408B
:102710000B43134308242343436110BD416908223E
:102720009143416170474269520852000A43426135
:10273000026801231B061A430260704701680122E8
:10274000120691430160704730B50C46124DA84205
:1027500001D1134D00E0184D2946184D4D60002B56
:1027600001D0202500E000254D61154D056030BDEC
:1027700001680122D204914301607047C269520886
:1027800052000A43C2617047C26916239A430A4342
:10279000C2617047F0430000000001400002005099
:1027A00000010140000011402800002040420F00BD
:1027B00000CA9A3BEF8FFFFF00011140FFFFFF00AF
:1027C0000000084070B5034600200FE0012484405B
:1027D0000C40002C09D01C6846000325B540AC43D2
:1027E00046001546B5402C431C60401C1028EDD314
:1027F00070BD10B58469130E8B401C438461C3699E
:102800001402240A8C402343C36110BD8269012352
:102810008B409A438261C369024A8A409343C361F1
:10282000704700000100010070B58C000459342588
:10283000AC4315461D43012635432C438D004451BE
:1028400070BD8A008258520852008B00C2507047F7
:1028500070B52F48006945076D0F00F020F82D492D
:102860000860022D03D0A8002B490C5801E029482C
:102870000468274880690007000F461C314620463F
:1028800000F08EF8254908602549244800684A1060
:10289000801800F085F82349086070BD7047FEB5C8
:1028A0000020029020A0006800901948046A0013DC
:1028B0002040002801D00020FEBD0120C00420409F
:1028C000002801D0194D00E0194D0120400420409E
:1028D000002801D02846EFE7032080032040800B2A
:1028E00069460A5C0192E005C00D861C1F2040026B
:1028F0002040400A871C019A7A431146AA08724375
:10290000104600F04DF8800002900298D4E70000D5
:102910000002005030000020104400002800002079
:1029200040420F002C0000200102020400805101EF
:10293000001BB7000748804707480047FEE7FEE74F
:10294000FEE7FEE7FEE7FEE704480549034A054BBC
:10295000704700009D280000C1000000A00000207A
:10296000A0040020A00000207CB51D4616460C00E7
:10297000009001D00019401E084B7B442A4669464E
:102980000190304600F06DF9002C054603D06946F1
:10299000002000F079F928467CBD000015030000F6
:1029A000002203098B422CD3030A8B4211D300234C
:1029B0009C464EE003460B433CD4002243088B4226
:1029C00031D303098B421CD3030A8B4201D39446B3
:1029D0003FE0C3098B4201D3CB01C01A52418309A6
:1029E0008B4201D38B01C01A524143098B4201D360
:1029F0004B01C01A524103098B4201D30B01C01A8B
:102A00005241C3088B4201D3CB00C01A5241830804
:102A10008B4201D38B00C01A524143088B4201D331
:102A20004B00C01A5241411A00D201465241104691
:102A300070475DE0CA0F00D04942031000D3404206
:102A4000534000229C4603098B422DD3030A8B423C
:102A500012D3FC22890112BA030A8B420CD38901DA
:102A600092118B4208D3890192118B4204D38901C0
:102A70003AD0921100E08909C3098B4201D3CB01FE
:102A8000C01A524183098B4201D38B01C01A5241B3
:102A900043098B4201D34B01C01A524103098B42B7
:102AA00001D30B01C01A5241C3088B4201D3CB00A2
:102AB000C01A524183088B4201D38B00C01A524185
:102AC000D9D243088B4201D34B00C01A5241411A5C
:102AD00000D20146634652415B10104601D340428A
:102AE000002B00D54942704763465B1000D340423B
:102AF00001B50020C046C04602BD70477047704710
:102B000070B5044685690068C10601D5302600E02D
:102B10002026C00707D070BD62683046A168904784
:102B2000206A401C20626D1EF6D570BD70B504464B
:102B300085690078C00707D170BD6268A168202050
:102B40009047206A401C20626D1EF6D570BD096852
:102B50004A0501D540B27047C905FCD500B270479F
:102B600009684A0501D5C0B27047C905FCD580B2D5
:102B7000704770B50C460546012A05D028788006B6
:102B800000D5EA69002302E0012305E05B1C9342C3
:102B900002D2E05C0028F9D1A869E618C01AA86141
:102BA000286AC01828622846FFF7AAFF04E06A686E
:102BB0002078A968641C9047B442F8D32846FFF7F0
:102BC000B5FF70BDF7B5002575291068009914A6EA
:102BD00011D0FFF7BCFF002802DA404211A608E03E
:102BE000009909688A0701D50FA602E0490704D5B4
:102BF0000EA6012501E0FFF7B3FF009F0024243754
:102C000004E000F01DFD30313955641C0028F8D176
:102C10002B4632462146009800F05FFAFEBD0000C8
:102C2000000000002D0000002B000000200000002C
:102C300011680268006A530501D5087009E0D305E0
:102C400001D5088005E0130602D5C21705C100E0D2
:102C5000086001207047000001694A1C0261087881
:102C6000704700B58FB0029100210591054901938D
:102C70007944039111460490684600F02DF90FB095
:102C800000BD0000E5FFFFFF0A681070521C0A60DB
:102C900070470CC908399A4202D2531C0B6010705D
:102CA00070470000F7B50446154686B02B487844B7
:102CB000002703C83E460090019111E007986A463C
:102CC0007100415A02A800F09BFC411C07D02178FA
:102CD000890603D5E269391891420ED83F18761C4F
:102CE0002078800602D5E069B84206DDAE42E5DB19
:102CF00007987100405A0028E0D1A069C01BA0616C
:102D00002046FFF7FDFE154878445A3803C8009066
:102D10000020019116E041006A460798415A02A836
:102D200000F06EFC0590401C0AD0002505E06268AA
:102D300002A8A168405D90476D1C05988542F6D3B6
:102D40000498401CB0420490E5DB206AC019206260
:102D50002046FFF7EBFE09B0F0BD00007E17000033
:102D6000F7B5D21D0025D20815A6D200F52905CA4F
:102D700011D0002A05DA00214042914111A60A46ED
:102D800008E0009909688B0701D50FA602E0490702
:102D900001D50EA601251146009F0024243704E02A
:102DA00000F05EF930323A55641C02460A43F7D10E
:102DB0002B4632462146009800F08FF9FEBD0000F8
:102DC000000000002D0000002B000000200000008B
:102DD00070B504460021243408E05507D2086D0F71
:102DE000303565545D072A43DB08491C15461D43F1
:102DF000F3D10468002310A2250708D5A40601D446
:102E0000002904D0C46901230CA2641EC46100F02F
:102E100064F970BD10B5044621461068FFF7A0FEA6
:102E2000002302462046FFF7D3FF10BDD21DD10874
:102E3000C9000CC9CCE70000000000003000000011
:102E4000F8B50F460188090502D5224C7C4402E002
:102E5000204C7C440E3405460021243508E016073A
:102E60001209360FA65D6E541E0732431B09491C1A
:102E700016461E43F3D1224604780023240705D5C5
:102E8000702F06D0002901D00223113200F025F95D
:102E9000F8BD01231032F9E770B504460D4621460E
:102EA0001068FFF75DFE0023024629462046FFF723
:102EB000C7FF70BDD21DD308DB000CCBC0E730B418
:102EC000036820241268234303600823C36130BCD5
:102ED0000023B5E7E8150000F3B50446002081B0F3
:102EE00020622046E1688847002872D0252802D059
:102EF0006268A168ABE0594F00267F442046E16834
:102F000088472028054608DB312D06D2781920385D
:102F10000078002801D00643F0E7B00701D504206F
:102F200086430020E0610746A0612A2D0AD028468A
:102F300001F0B4F9002827D0B8000019303D009006
:102F4000856119E00298BA00121902C891610290D5
:102F50002046E1688847012F054617D1E06900281F
:102F60001FDA202086431CE000980A21806948432C
:102F700000994019303888612046E1688847054645
:102F800001F08CF90028EFD1012F0AD02E2D08D1A5
:102F90002046E16888470546202006437F1C022F13
:102FA000C3DBA069002803DA4042A0610120064388
:102FB000F00701D0102086436C2D0BD0682D09D06E
:102FC0004C2D3CD06A2D38D0742D38D07A2D36D087
:102FD00016E040E0E1682F4620468847B8420546A3
:102FE00009D16C2F29D001208002E16806432046D8
:102FF0008847054604E06C2F1DD0FF2001300643B2
:10300000002D28D028464138192803D80120C002B5
:1030100006432035204626602946029A1646FDF7CB
:103020008DF8002810D001280BD0F61DF008C00044
:103030000830029055E74020E1E78020D5E70020E6
:10304000D3E7361D02964CE762682846A168904790
:10305000206A401C44E7206AFEBD000062150000A3
:103060000B4670B5024689078008084319469D083B
:10307000141AA94125090807054308092C194841D4
:10308000250A01060D43010A2C194141200C0D04AB
:1030900028430D0C00194D41002140194D41C00835
:1030A00069070843E908840F8D002543840024182C
:1030B0004D4124196D41121BAB4107E00925ED4339
:1030C0002C11521963410024401C61411C460A2501
:1030D0000026551BB441F1D270BDFFB504460D4624
:1030E00081B0243000902168880604D51022E06960
:1030F0009143216000E00120A84201DD471B00E070
:1031000000270498A1697A191018081AA06120787C
:10311000C00602D42046FFF7F3FC002608E003981F
:103120006268A168805D9047206A401C761C20621E
:1031300004988642F3DB2078C0060AD52046FFF7C4
:10314000DFFC06E06268A16830209047206A401CDE
:10315000206238467F1E0028F4DC07E00098626891
:10316000A168405D9047206A401C206228466D1E81
:103170000028F3DC2046FFF7D9FC2078000602D5B2
:10318000022005B0F0BD0120FBE700007047FFB54D
:103190000C461E468FB003CA089009914F007D0D62
:1031A00000D16D1E002108460020C0460321099A67
:1031B00089050840002A03DA820080184008084088
:1031C000800D01280A9002DD0020C0430A90089873
:1031D00007430DD0F048F1492818484307141898C0
:1031E00000281DD07542291E1DDD0A9842421BE0B1
:1031F0001898012802D00020302104E00020F2437A
:1032000005E02154401CB042FBDB30460022189BF5
:10321000002121540F998B600A60486013B0F0BD03
:10322000BD1B6D1CDFE70A9A002900DA69420BA872
:1032300000F08AFA0BAB07CB03AB07C308990998D8
:1032400000F0EEFA6B4607C30146D5480918002D79
:1032500000910BDDD24903980A9A49424018002395
:1032600003A90390684600F04BFD08E003990A9A11
:103270000023081803A90390684600F0EBFC6B4696
:1032800007C30004000C03D00020C043410800E045
:103290001046189A002A03D00022009215461EE01C
:1032A000751E05D4FFF7DCFE303262556D1EF9D570
:1032B00001220843079602D000227F1C04E02078F8
:1032C000302801D100227F1E002A069787D01EE0F9
:1032D000112D07DAFFF7C4FE303262556D1C02462D
:1032E0000A43F5D1084303D00098002819D00EE016
:1032F0000021681E05E0235C625C63542254401E7A
:10330000491C8142F7DBA81B401E07950690079ACF
:1033100018990020A0540F98079B069A81600CC052
:103320007CE711260020189059E7D21DF0B50D4614
:103330000446D10893B0C90003C90C900D9100F068
:1033400097FF02460D98C00F01D02D2007E020689E
:10335000810701D52B2002E04007C00F4001032A5E
:103360000F9001D0072A05DB03462946204600F0CE
:10337000A7F90EE12078800601D5E76900E006276D
:103380002846652D04D0662814D0672D69D12DE01C
:103390000020112F009001DB112300E07B1C0CAA00
:1033A00003A910A8FFF7F3FE1199002610987D1CC1
:1033B0000E9142E001203B460CAAC0070B90012071
:1033C000009003A910A8FFF7E2FE119D1298109932
:1033D000002600280E9501D1781C0D18781B02D408
:1033E00046427D1C761EE81B00903AE0012F00DA71
:1033F00001270020112F009001DD112300E03B4642
:103400000CAA03A910A8FFF7C2FE11993D46109817
:1034100000260E91217809070BD40E99A94200DAF3
:103420000D4603A9012D04DD4A19203AD27F302A26
:1034300006D0B84201DA011D04DA012100910FE043
:103440006D1EEFE7002802DC86192D1A03E0411CEF
:10345000A94200DD0D46801B401C00900120C007E2
:103460000B902078000705D40098A84202DB0020CA
:10347000C043009069460020C8720B98012102AF3A
:103480000337C907884225D0022010902B201190C5
:103490000B9800280BDA40420B902D20119006E08B
:1034A0000B9800F0CDF830317F1E0B9039701099D9
:1034B000481E00291090F3DC0B980028F0D11198D9
:1034C0007F1E38702088000501D5452000E065206A
:1034D0007F1E387001A8C01BC01D0B900F980028DC
:1034E00000D0012041190098C01709180B9808183E
:1034F000A169081A401EA0612078C00602D42046A7
:10350000FFF7FEFA0F98002805D06268A16890477F
:10351000206A401C20622078C00625D52046FFF78F
:10352000EFFA21E0002E07DB0E98B04204DD03A87D
:103530006268805DA16802E06268A16830209047FF
:10354000206A761C401C20620098401E00280090D3
:103550000AD100F0B1F8C06862680168405CA168F7
:103560009047206A401C206228466D1E0028D9DC46
:1035700007E062683878A1687F1C9047206A401C89
:1035800020620B99481E00290B90F2DC2046FFF7C1
:10359000CDFA032042E6000001FCFFFF104D0000C1
:1035A000E1DFFFFF10B54369002B02D0C046C046E3
:1035B00001E0FFF7DEFA012010BD12780146243148
:1035C0000A7000224A700122ECE711680022D243FF
:1035D000E8E710B54369002B02D0C046C04601E0C1
:1035E000FFF760FB012010BD128801462431828460
:1035F0000022C2840122ECE711680022D243E8E7EE
:1036000070B516460C46054600F04EF80368FF20DC
:103610000230C05C012807D0FF2C0ED8185D0028AE
:103620000BD001202C7070BDFF3332462146083389
:103630001868C3182846984770BD0020C04370BD65
:1036400001468008081A02091018020A1018020C14
:103650001018C008820012185200891A01E0401C9C
:103660000A390A29FBD27047754600F0A1FBAE4625
:10367000050069465346C008C000854618B020B50D
:10368000FFF762F960BC00274908B6460026C0C5AE
:10369000C0C5C0C5C0C5C0C5C0C5C0C5C0C5403D0A
:1036A00049008D467047000010B500F005F8001D78
:1036B00010BD00BF250C00000048704760000020CE
:1036C000F8B51F46044601230068DB0203260146C5
:1036D0001840072A05DB002801D017A506E017A52A
:1036E00004E0002801D016A500E016A510208143B3
:1036F0002160A069C01E002FA06101D0401EA06102
:103700002046FFF7FDF9002F09D038466268A1680E
:103710009047206A401C2062C01C206206E0206A9C
:10372000FAE762682878A1686D1C9047761EF8D287
:103730002046FFF7FBF9F8BD4E414E006E616E006A
:10374000494E4600696E6600F7B516468AB03348A2
:1037500078446C4603467C33C06F5A689B680DC43E
:103760002E487844763003AC0DC80DC43720C00114
:10377000081837211B30FFF71DF905460C46803D20
:103780001B3C02D56442012000E000200027099084
:1037900010E0E0070CD00C202049784379443246F1
:1037A0004C3941186846012300F054FA6B4607C3B0
:1037B00064107F1C002CECD1184F7F442E3F16E084
:1037C000E80712D02001C0190EC80691089307928D
:1037D0000068F04201D1981908903246012306A9E9
:1037E00003A800F037FA03AB07C36D10641C002D6B
:1037F000E6D10998002806D032466946012303A87D
:1038000000F07EFA05E001233246694603A800F085
:1038100021FA0A9B07C30DB0F0BD0000200D000087
:10382000034640000A4610B5400D0BD00121C907E0
:103830000F24A40200191C0364082143540D2143E2
:10384000D20207E000210120F2E7D40F4900214312
:103850005200401E0029F8DADB0FDB07184310BDC9
:10386000FFB50D46144685B04868516800F0DAFC93
:1038700000910190A868A16800F0D4FC0291039027
:10388000A868616800F0CEFC029A12188242029287
:1038900001D2012000E00020019A0B18D218002864
:1038A000019202D08A4202D903E08A4201D2012069
:1038B00000E000200099081800906868A16800F0F6
:1038C000B1FC029A12188242029201D2012000E059
:1038D0000020019A0B18D2180028019202D08A42C7
:1038E00002D903E08A4201D2012000E000200099C1
:1038F00008180090286821684000490040084908DD
:103900004018FA49471814E001994000C90F0843CC
:103910000090019802994000C90F08430190029855
:1039200003994000C90F08430290039840007F1E8E
:10393000039000980028E7DA0898002801D0EC4EA0
:1039400000E00026B74201DA012000E00020002854
:1039500004902AD0F71BF806C00E15D0029B202138
:10396000091A039A8B401A430392029A019BC240A0
:103970008B401A430292019A009BC2408B400099EF
:103980001A430192C14000917B110DD06F46032074
:10399000C11A03D500218200B95003E08A008100DA
:1039A000BA587A50401EF3D537460398029900283A
:1039B00000D00120014308980291002808460CD04D
:1039C000002800D001200199019A490508430121EE
:1039D000D20AC902D202019200E001210E9B01220B
:1039E000D207012B02D0002B03D013E0002807D10F
:1039F00020E0904204D890420CD1019B0B4209D0A8
:103A0000019B5918019105D10099491C009101D1E0
:103A10007F1C009200280DD0102108460020C046CF
:103A20000498002806D00F98002803D008210846E3
:103A30000020C04628682168019B009A4840C10FB9
:103A40000598C90739430EC009B0F0BDFFB587B06E
:103A5000099A089808995368926840688968964658
:103A60000022039317469446089A12685300099A55
:103A70005B081268520052089A1A9E4BD4180A9A90
:103A8000002A01D0352200E04022069200220123C4
:103A900015460492DB07059324E0002D05D17546F9
:103AA0000346039E4D1BB34109D375466646039BEF
:103AB000491B049D9841059B7519AC465F416346BF
:103AC0003B4308D0059B049EDD0776082E435B0828
:103AD0000496059301E0521E641EC50FED074918B8
:103AE0004041521C069B9A42D7DB002D04D17546FB
:103AF000039A6B1A824101D203200CE0039A0B4611
:103B00006B404240134303D0014303D0012002E045
:103B1000022000E0002061460191002100970291FF
:103B20000A99002905D0614640020143704B01917A
:103B300002E08007002302909C4201DA012000E0AD
:103B4000002007003AD01A1BD006C00E15D0029DE7
:103B50002021019C091AC5408C402543029C8C40C1
:103B600000D001242543019C0295009DC4408D4056
:103B700000992C430194C140009154111DD06D4611
:103B80000221002202290CD10320001B07E000289B
:103B900004DB8600AE59002E00D00122401C032811
:103BA000F5DB081B02D588002A5004E08000285865
:103BB00010438A00A850491EE3D51C460A980028E5
:103BC00002980CD0002800D001200199019A4905E3
:103BD00008430121D20AC902D202019200E0012168
:103BE000109B0122D207012B02D0002B03D013E03F
:103BF000002807D11FE0904204D890420CD1019BCD
:103C00000B4209D0019B5918019105D10099491C1B
:103C1000009101D1641C009200280CD010210846AC
:103C20000020C046002F06D01198002803D008219C
:103C300008460020C04608980999019A009B006830
:103C400009684840C10F0798C907214382600AC02C
:103C50000BB0F0BD00B585B0019300920A46014655
:103C6000002302A8FFF7FCFD02A807C805B000BDAD
:103C7000FFB50A461F4685B00799019301230091BD
:103C8000014602A8FFF7ECFD02990398049ECA0FB3
:103C90004900D20700920F22490892028C1A002193
:103CA000002800DB0C46450013486D08844214D3FD
:103CB000079A002A04DA441E0026104DF64302E05B
:103CC00004460D460E46102108460020C046002F2F
:103CD00003D0042108460020C0462005E90A084315
:103CE000009908436905F20A1143ADE602C0FFFFDF
:103CF000013C0000FF3F0000FF070000FFFFFF7FC7
:103D000000B585B0019300920A460146002302A83F
:103D1000FFF79CFE02A807C8A8E7FFB50A461F46A2
:103D200085B00799019301230091014602A8FFF78E
:103D30008DFE02990398049ECA0F4900D207009293
:103D40000F22490892028C1A0021002800DB0C4641
:103D5000450011486D08844214D3079A002A04DAFA
:103D6000441E00260D4DF64302E004460D460E4665
:103D7000102108460020C046002F03D00421084629
:103D80000020C0462005E90A084300990843690558
:103D9000F20A114358E60000FF070000FFFFFF7F13
:103DA00010B50446C046C0462046FCF753FA10BD85
:103DB0000048704740000020024670B50A43920751
:103DC0002AD11E4DEE0104C808C9541B9443344047
:103DD00017D0D0B2D9B2401A2106014310D190B207
:103DE00099B2401A210401430AD110021902000AB3
:103DF000090A401A2102014302D1100E190E401A7D
:103E000070BD9A42DFD010BA19BA884201D9012098
:103E100070BD0020C04370BD02780B78401C491C67
:103E2000002A09D09A4207D102780B78401C491C1D
:103E3000002A01D09A42EFD0D01A70BD01010101D1
:103E400001491820ABBEFEE72600020070470000C3
:103E500010B577480068401C75490860322807D3C0
:103E6000002008607349C86372494039486205E020
:103E700001207049C8636F49403948626E48006844
:103E800000281DD06B48006900280BD069484069A4
:103E9000002807D067488069002803D06548C069BA
:103EA000002803D10A2065490860C0E06348006823
:103EB000401E624908600028F7D15F490860B6E0FB
:103EC0005C48006900280FD101205B4908600A2086
:103ED0005A4908605A480068401E5949086000283D
:103EE000E3DA00200860A2E05248406900280FD1C0
:103EF0000120514908600A20504908605048006874
:103F0000401C4F4908600628CFD3052008608EE08A
:103F10004848C069002843D10120474908600A2069
:103F200046490860464800688000464908584649A6
:103F30000968081A444908600846006843498842ED
:103F400003DA0846404908600CE041480068401E1A
:103F50003F490860302801DA392008603C49087878
:103F6000FCF714FE38490C68E10F09194910394A69
:103F7000881835490968FEF713FD401E2C49086072
:103F8000084601680020FCF755FC2948016802201A
:103F9000FCF750FC264801680420FCF74BFC46E087
:103FA00024488069002842D10120234908600A2062
:103FB00022490860224800688000224908582249A6
:103FC000096840182049086008460068224988426C
:103FD00003DD08461C4908600CE01D480068401CD1
:103FE0001B490860392801DD30200860184908782D
:103FF000FCF7CCFD14490C68E10F09194910154A6A
:10400000881811490968FEF7CBFC401E0849086072
:10401000084601680020FCF70DFC054801680220F5
:10402000FCF708FC024801680420FCF703FC10BD03
:1040300038000020C04200503C0000203400002026
:10404000040000201443000000000020409C0000F9
:104050000800002000A24A04F04902007CB569462D
:1040600001A8FCF732FE0546002D70D0642D25D046
:104070000CDC542D6CD004DC202D6AD0462D1CD1D4
:10408000B6E0562D7ED0612DF9D163E0762D7AD041
:1040900004DC662D07D0742DF1D1A7E0772D42D036
:1040A000782DECD18EE057480068800056490A58B8
:1040B000564801685648FCF7E3FDA0E05148006807
:1040C00080005149085851490968081A4F49086049
:1040D000084600684F49884202DA08464B490860A2
:1040E0004A490E68F10F891949104B4A8818474907
:1040F0000968FEF755FC441E21460020FCF79AFB98
:1041000021460220FCF796FB21460420FCF792FB97
:104110003C48006880003C490A583C4801683C48DB
:10412000FCF7AEFD6BE037480068401E354908607B
:10413000002801DA00200860324800688000324917
:104140000A58324801683248FCF79AFD57E057E0B8
:104150004FE050E02B48006880002B4908582B495D
:104160000968401829490860084600682B498842B8
:1041700002DD08462549086024490E68F10F8919B7
:10418000491001E036E032E0234A88181F490968E7
:10419000FEF706FC441E21460020FCF74BFB21469F
:1041A0000220FCF747FB21460420FCF743FB15489F
:1041B0000068800014490A58144801681448FCF744
:1041C0005FFD1CE00F480068401C0E49086006288F
:1041D00001D3052008600B48006880000A490A588E
:1041E0000A4801680A48FCF74BFD08E000BF00BF21
:1041F00000BF00BF00BF0A48FCF742FD00BF00BF80
:104200007CBD0000040000201443000000000020DA
:1042100008450000409C000000A24A04F04902004A
:1042200027450000F8B5040C8BB2264682B25E43E7
:10423000104658430D0C370C3604002180191646E1
:1042400079416E43370C36048019264679416E4316
:104250008919F8BD30B47446641E2578641CAB42DD
:1042600004D3635D5B00E31830BC18471D46F8E7D4
:104270004900CA020243100000D004204A0D01D0B8
:1042800001221043044A490D914201D10221084301
:10429000012800D105207047FF07000030380A28A8
:1042A00001D20120704700207047000010B500299E
:1042B0000AD00878002807D005487844FFF77CFD2D
:1042C000002801D0002010BD0248784410BD000035
:1042D000920200008A02000010B500290AD0087876
:1042E000002807D005487844FFF766FD002801D074
:1042F000002010BD0248784410BD0000820200007A
:104300007A02000003B402487844844603BC604744
:104310001FF0FFFF1027000088130000E8030000D3
:104320006400000019000000050000000030224178
:104330006D527C20390F2170084080523F065B4F40
:10434000666D7D077F6F484839480F535F777C392A
:104350005E79713D76061E763815373F7367316D8D
:10436000786E1C2A766E5B39640F230820777C58A0
:104370005E79716F74041E761815545C7667506D03
:10438000783E1C2A76675B466E3D6D6E6E000000BF
:1043900000000000040000000C00000024000000E9
:1043A00000000000200000000000000004000000E9
:1043B0002C00000000000000040000002C000000A1
:1043C000001BB700000000000080000000805101C9
:1043D000001BB700000000000080000000805101B9
:1043E000001BB700000000000080000000805101A9
:1043F000001BB7000080000000000000000000006B
:1044000000000000102700000000000000805101A3
:10441000001BB7000080000000E0480410270000E7
:10442000006CDC0200000000000000000080510170
:1044300000000000000000003031323334353637E0
:1044400038394142434445464030580030313233D8
:1044500034353637383961626364656640307800D8
:10446000040000080000000000000002000100003D
:104470001000000002400000000000A0000000004A
:1044800005400000000000C8000000000C400000D3
:104490000000409C00000000194000000020BCBE4D
:1044A0000000000034400000BFC91B8E0000000463
:1044B000B5400000504BCFD06607E2CF01000000AE
:1044C0006C4100003E8251AADFEEA73401000000DB
:1044D000D9420000DCB5A0E23A301F97FFFFFFFF92
:1044E000B4450000FD25A0C8E9A3C14FFFFFFFFFB1
:1044F000FF3F00000000008000000000FF3F0000C0
:104500000000008000000000437572724672657101
:10451000203D2025642044656C74614672657120DD
:104520003D2025640D0A004E410D0A00784600002A
:10453000000000204000000004010000B846000018
:104540004000002060040000200100001C0000006A
:1045500043000000F8FFFFFF0C0000000E00000009
:104560000F0000002E0000001001000043000000BA
:10457000F8FFFFFF00404040404040404040414184
:104580004141414040404040404040404040404028
:1045900040404040400502020202020202020202C2
:1045A00002020202022020202020202020202002BF
:1045B000020202020202909090909090101010104F
:1045C00010101010101010101010101010101010EB
:1045D000020202020202888888888888080808087F
:1045E000080808080808080808080808080808084B
:1045F0000202020240000000000000000000000073
:1046000000000000000000000000000000000000AA
:10461000000000000000000000000000000000009A
:10462000000000000000000000000000000000008A
:10463000000000000000000000000000000000007A
:10464000000000000000000000000000000000006A
:10465000000000000000000000000000000000005A
:10466000000000000000000000000000000000004A
:104670000000000000000000F049020000000000FF
:104680003000000000000000FFFFFFFF00000000FE
:10469000000000000000000000000000000000001A
:1046A00000E048044700000000E04804000000006B
:0846B000000000000000000002
:040000050000293599
:00000001FF
